:030000000219FDE5
:03000B000200A848
:03002B0002015A75
:03005B000202EEB0
:030073000202DBAB
:1000800002030406080C10182030406080040608A3
:100090000C10182030406080A0C00003070F1F051F
:1000A000050D050305030302C2AFC0D0C0E0206206
:1000B00014E5256009E473E525F4F58AD262D0E001
:1000C000D0D0D2AF3285268AC262E526F4602F30C6
:1000D000682520720DD0E0D0D0D292D291D290D2A9
:1000E000AF32D292D291D290206F0C206609740A5E
:1000F000D5E0FDE57B4290D0E0D0D0D2AF32758A1A
:1001000000C28DD26201F701B7306805206602C2D5
:100110009201B7306805206602C29101B7306805C8
:10012000206602C29001B7C29330680A2066077445
:1001300008D5E0FDC29201B7C29430680A20660774
:100140007408D5E0FDC29101B7C29530680A2066F7
:10015000077408D5E0FDC29001B7C2AFC2AD53E647
:10016000EFC0D0C0E0D2D3D2AFC2CEE52A60072024
:100170007449152A21BB7800790020742EE580305F
:100180007E01F430E40278FF53DACF207E0343DAB5
:1001900020307E0343DA10C2D8C271E580307E0180
:1001A000F430E40279FFC3E89970CB306103752A1B
:1001B00018207403752A18885CD27020740DE52B02
:1001C0006004152B21CB43DA01C2D8207002413ED6
:1001D000A85C206102C270207431C3E894F040032F
:1001E00074F0F8E8C4540F28F87984B70302410B7F
:1001F000C313C3138721200802C313200A06C3C8F0
:1002000098F8410B28F8500374FFF8C3E89565503F
:1002100003E565F88822E52D54066022206B1FE572
:1002200036C333C333F8E564C313C313F9C395224C
:1002300040028922E82522F52250037522FF8522FB
:1002400024A824C3E52495614002A8618825E566B9
:1002500070024182C3E8AA669A5003E8FAE4F9EA18
:10026000C333FBE568F45B29400D2567F8E567605B
:10027000021567400B41820AC3E5679A5002056781
:1002800078FF8826C26FC3E52694F84002D26FC378
:10029000E52594404002D26420CF0AD0E0D0D0437C
:1002A000E610D2AD32C2CF053A7801E52A600530BA
:1002B0007402152AC3E55C94014005755F0041D1C5
:1002C000756000756900E55F2401F55F5003755F97
:1002D000FFD0E0D0D043E610D2AD32C2AF53E67FBC
:1002E0007592FA7593FFC260759104D2AF32C2AFB6
:1002F00053E6EFC2ADC0D0C0E0C0F0D2D3D2AFA8B9
:10030000FBA9FCC2D8307102615553DACF207E03BD
:1003100043DA10307E0343DA20D271E580307E016B
:10032000F420E402612C88278928A18253DACF20A7
:100330007E0343DA20307E0343DA10C2D8C2713024
:100340007402A16E7800E580307E01F430E402A1F1
:100350006E885CA15653DACF207E0343DA20307ECC
:100360000343DA10C271206102812E53DACF207E5E
:100370000343DA10307E0343DA20C2D8D2718857A3
:100380008958C3E89555F8E99556F97B007E087AB7
:1003900000C3E8948CE994005005755B00812088C7
:1003A0002178A2E6A8216055C3E894C8E9940050DA
:1003B00008E4D2E4FB7A0A61FBC3E89468E994019B
:1003C0005008E4D2E3FB7A0F61FBC3E894D0E994D0
:1003D000025008E4D2E2FB7A1E61FBC3E894A0E974
:1003E00094055008E4D2E1FB7A3C61FBC3E89498A1
:1003F000E994085008E4D2E0FB7A787E00C3E895DF
:1004000059FCE9955AFD30E70AECF42401FCEDF4BF
:100410003400FD755B00C3EC9AED9E5003755B01E3
:100420008859895A8557558558567802A156C3E888
:100430009527F8E99528F9307C02A13A307B02A192
:100440003A307A02A1332075028151E9FDE8FC813E
:1004500070E9C313F9E813F8307902A133E9C31343
:10046000F9E813F8307802A133E9C313FDE813FC6F
:0F04700020612CC3EC941CED940240028187EDB7
:10047F00701EC3EC94C850180529E5297002152980
:10048F00C3E529940A5002A16E755C00D270A16E6B
:10049F00E529600215297888E6F97400207F08782D
:1004AF0096B90302789EE624FAFEE43400FFC3EC0B
:1004BF009EFCED9FFD9208B90310A208500720760D
:1004CF0009D27681D9307602C276A2085016B903C6
:1004DF000DECF42401FCEDF43400FD0204F378007C
:1004EF007900A13AB90315EC33FCED33FDC3EC945D
:1004FF000AFCED9400FD50047C007D00C3EC94FFDA
:10050F00ED9400400678FF7900A13AEC8572F0A4D3
:10051F00C5F0A2F733F87900400302055678FF794A
:10052F0000020556E9C313F9E813F8307C0EE960B1
:10053F000278FFC3E81338F8E43400F9C3E894FFF6
:10054F00E99400400278FF885CD270206102A16EAE
:10055F00741FF4552F4BF52FC274EB7002D27475C4
:10056F002A18307403752A0A306102A1822074039D
:10057F0053DAFE207403752B06D0F0D0E0D0D0D222
:10058F00AD43E6103279010205B279030205B27963
:10059F000A0205B2791E0205B279640205B279C862
:1005AF000205B27817E4D5E0FDD8FAD9F6227A140D
:1005BF007B780205D97A107B8C0205D97A0D7BB432
:1005CF000205D97A0B7BC80205D97902E4C294D50A
:1005DF00E0FDC291D5E0FDD291D5E0FDD294D5E0FA
:1005EF00FDE920E002C29230E002C290E573D5E04F
:1005FF00FDE920E002D29230E002D2907496D5E06D
:10060F00FDD9C9EAF8D5E0FDD8FBDBBEC29422C301
:10061F007C007D0075F00005F0EA33FAEB33FB50F8
:10062F00F6EB13FBEA13FAC3E9FFE8FEE89AF8E9E1
:10063F009BF95004EFF9EEF8B3EC33FCED33FDD535
:10064F00F0DFEDF9ECF822E889F08A20D2D4F8A98E
:10065F00F07B0030F70B7BFFF42401F8E9F4340052
:10066F00F9E88520F0A4ADF0F8E98520F0A4AFF00B
:10067F00FEED2EF974003FFA7C04C3EA13FAE91376
:10068F00F9E813F8DCF48BF030F70AE8F42401F8FA
:10069F00E9F43400F9E889F0C2D4F8A9F02222C3B2
:1006AF00E54113F9E54013F8C3E54498F8E545999A
:1006BF00F9500CC3E89480E994FF40160206E5C395
:1006CF00E8947FE9940050030206E5787F790002F1
:1006DF0006E5788079FF8849894A22E5492546F859
:1006EF00E54A3547F9854A20E4300701F43548FAE1
:1006FF0030E709C3EA94F04015020723C3EA940FC9
:10070F00500302072378FF79FF7A0F02072378003F
:10071F0079007AF0C3E5249561500AC374019524DA
:10072F00500B020741E54A20E70E020741E54A3028
:10073F00E706884689478A482278A5E6FAC3E5493D
:10074F0033F8E54A33F9D156E930E70BC3E8948023
:10075F00E994FF4013E17BC3E8947FE994005002D2
:10076F00E17B787F7900E17B788079FFE820E715DE
:10077F00C3E52398F84009C3E8940140030207A298
:10078F0078010207A2E8F424012523F840030207A9
:10079F00A278FF884B2278A6E6FAA847A948D15637
:1007AF00E930E70CC3E89401E994FF40160207D63D
:1007BF00C3E894FFE9940050030207D678FF79004D
:1007CF000207D6780179FFE920E715C3E54B98F8C2
:1007DF004009C3E8940140030207FD78010207FDB9
:1007EF00E8F42401254BF840030207FD78FF882425
:1007FF002278FFC26420693D206A12D264C3E541AA
:10080F00940A4009C3E52594405002C26479A1E7D8
:10081F006023E541601F74FF8541F0848539F03016
:10082F006A0375F005A4F8C5F0600278FFC3E89578
:10083F00645002A864886322C3E5409440E5419464
:10084F0001E5635003140158046002F563220208A6
:10085F00602275E890227883E6FFE5E820ECF7A8A0
:0F086F00BDA9BE0570C3E57094084052757000B6
:10087E00E9FA79A0E76044EA7007E571601B0208A7
:10088E009BC3E895716010E5715006600C14020868
:10089E00A70460F90208A7E571F571C39458401BCF
:1008AE007561C0C394044013756180C39404400BFA
:1008BE00756140C39404400375610075BB0322E566
:1008CE0061F460020561E570B4070375BB10227414
:1008DE003279A787F0A4C5F0A2F733F8C3E8956183
:1008EE004002A8618822882488258826886422757B
:1008FE0040007541F022C2AF75C820A8CCA9CDAA80
:10090E003A30CF010A75C824D2AFAB3BAC3C883B22
:10091E00893CC3E89BF8E99C206908F930670241DD
:10092E0010216DAD3D8A3DF9EA9DFA600478FF799C
:10093E00FFAE3EAF3F8B3E8C3FA83BA93CC3E89E2B
:10094E00F8E99FF9C3E54113FBE54013FAE82AF5F0
:10095E0040E93BF54150067540FF7541FF21B7AAAE
:10096E0040AB41AC40AD417E047F02C3EB940440EA
:10097E00021E1FC3EB940840021E1FC3ED13FDECB5
:10098E0013FCDEF7C3EA9CFAEB9DFBEF6009C3E9AB
:10099E0013F9E813F8DFF7EA28FAEB39FB8A408BF4
:1009AE004150067BFF8B408B41C3EB94025002D229
:1009BE00673069047F0321E27892E6FFC3E537943E
:1009CE008240110FC3E53794A040010FC3EF940688
:1009DE0040027F057E02E541C4540FF9E541C4543F
:1009EE00F0F8E540C4540F28F8C3E89EFAE99400E5
:1009FE00FB4009C3EA9402EB940050047A02E4FB34
:100A0E00415CAA40AB41EBC4FEEAC4540F4EFCC39A
:100A1E00EA9CFAEB9400FBC3E813C313F8EA28FA36
:100A2E00EB3400FB8A408B41C3EB94024002C26759
:100A3E007802EBC4FE7B00EAC4540F4EFAC3EA9868
:100A4E00FA4005C3940250027A027892E6FF3060B3
:100A5E0002415C855192855293D26043E680C3E495
:100A6E009AF8E49BF930670241E8E8FAE9FBD3E92A
:100A7E0013FDE813FC88518952C3EF94036038EFDD
:100A8E0020E00DE82CF8E93DF9ECFAEDFB020AB195
:100A9E00E828F8E939F9C3E82402F8E93400F97ACC
:100AAE00FE7BFFC3EF9403400E8A538B54884D890F
:100ABE004E8C4F8D50611C885389548A4D8B4E8CB1
:100ACE004F8D503069127553F07554FF754FF07598
:100ADE0050FF7551F07552FF611CE8FAD3E813FC14
:100AEE008851C3EF94036020EF20E007E82CF8EC68
:100AFE00FA6108E8282402F87AFEC3EF940340084E
:100B0E008A53884D8C4F611C88538A4D8C4FE568F3
:100B1E00C3335002646BF56830600261267534028F
:100B2E00D26043E680E52D54066034A840A941C347
:100B3E00E913F9E813F8C3E913F9E813F830690477
:100B4E00E92440F9C2AF53E67F759100C3E498F5EE
:100B5E0094E499F595759104D26043E680D2AF2264
:100B6E00D265754300752000306C03752040020B72
:100B7E008DD265754300752040306C03752000786A
:100B8E00017901206720E52D54066002C2657914B3
:100B9E00E541C313700104F8C39414400278143075
:100BAE006904781B791B206010E543600C306903E3
:100BBE00D53404D26D8130712E0543E59BF454403B
:100BCE00B52002811A30690908C3E89940011861FD
:100BDE00B420650A08C3E8994002618D61B4C2650C
:100BEE00C2AF53E67F75910030671275940075950C
:100BFE00FE759104D26043E680D2AF618DAE40AFF8
:100C0E0041C3E49EF594E49FF59561FFC3E53394EB
:100C1E00015002618D306502618DD802812E61B462
:100C2E00C26DC2AF53E67F7591008553948554957E
:100C3E00759104854D92854E93D26043E680D2AF76
:100C4E00E52D54066008206A020533020C6C306DE7
:100C5E000D206C0A2065071581158102151A227860
:0F0C6E00003064053065027801E53775F007A4A2
:100C7D00F9E5F028F5F0E9A2F013A2F113A2F213B1
:100C8D00F537C394785003753778C3E537953840F9
:100C9D0008D266D292D291D29030600281A6854F51
:100CAD0092855093D26043E68022D2A0207D16C259
:100CBD00AF754202C294D293306202C290D2AF7528
:100CCD009F10020EB2C2AF754202C294D29530622D
:100CDD0002C292D2AF759F10020EB2C2A030724303
:100CED00207D20C2AF754203900138757B10D290E4
:100CFD00C295306204C291A108D294D2AF759F20E3
:100D0D00020EB2C2AF754203900138757B10D292BC
:100D1D00C293306204C291A128D294D2AF759F00C4
:100D2D00020EB2207D17C2AF754203900113D2900F
:100D3D00306202C291D2AF759F20020EB2C2AF7562
:100D4D004203900113D292306202C291D2AF759FCD
:100D5D0000020EB2D2A0207D16C2AF754204C2931E
:100D6D00D295306202C291D2AF759F00020EB2C20F
:100D7D00AF754204C295D293306202C291D2AF7563
:100D8D009F20020EB2C2A0307243207D20C2AF75EB
:100D9D004205900127757B08D291C294306204C23E
:100DAD0092A1B2D293D2AF759F10020EB2C2AF759F
:100DBD004205900149757B20D291C294306204C2E4
:100DCD0090A1D2D295D2AF759F10020EB2207D1791
:100DDD00C2AF754205900109D291306202C292D222
:100DED00AF759F10020EB2C2AF75420590011DD2B4
:100DFD00913062EBC290D2AF759F10020EB2D2A0AD
:100E0D00207D16C2AF754206C295D294306202C2E1
:100E1D0092D2AF759F20020EB2C2AF754206C29339
:100E2D00D294306202C290D2AF759F00020EB2C250
:100E3D00A0307243207D20C2AF75420190014975EB
:100E4D007B20D292C293306204C290C15CD295D203
:100E5D00AF759F00020EB2C2AF75420190012775AA
:100E6D007B08D290C295306204C292C17CD293D2DB
:100E7D00AF759F20020EB2207D17C2AF7542019053
:100E8D00011DD292306202C290D2AF759F00020E48
:100E9D00B2C2AF754201900109D290306202C29286
:100EAD00D2AF759F20C26622900107757B00D2924A
:100EBD00D291D290C293C294C295C26222788076AA
:100ECD00FF0876FF0876FF0876FF0876030876049C
:100EDD0008760A087603087601087601788C760183
:100EED000876FF0876FF0876FF0876FF0876FF087C
:100EFD0076030876FF0876FF0876FF0876250876D4
:100F0D00D00876FA0876FA0876040876FF08760196
:100F1D0008760008767A0876FF08760108760108CB
:100F2D007600087603087600227887E6FFC272BF46
:100F3D000302D2727888E6C394036008C27DE6305E
:100F4D00E102D27DC27E7889E630E102D27EC3EF26
:100F5D0094026008758E01D273020F6E758E00C2F9
:100F6D0073227880E6149000809378A5F67881E658
:100F7D00149000809378A6F67886E61490008D93F1
:100F8D0078A7F67886E6F539C394025003753902D1
:100F9D00789CE67538FFB402037538A0B403037569
:100FAD00388278A3E61490009A93F566D1B5222283
:100FBD007896E6FA7897E6FB7888E6B40305C3EBF6
:100FCD00940EFB307F047A007BFFC3EB9AFCC39435
:100FDD008250027C827572000572EC8572F0A4C39A
:100FED00E5F0947D40F222D27FF1BD1205A37A0087
:100FFD007B007C10120599E55C2AFA74003BFBDC42
:10100D00F37C04C3EB13FBEA13FADCF7FEC27F1289
:10101D000FBD22E5EF20E6037520000520903FFF70
:10102D00E520146006901DFF1460009304600375A5
:10103D00EF1253D9BF7581C043FF8012059475EF30
:10104D000243B203E5B3240220E70DF521E5E320C9
:10105D00E0068521B343E301120EB57580FF75A43B
:0D106D000075F1D475D4EF75908775A5401E
:10107A0075F2FF75D5BF75A60175E24275DB467537
:10108A00EA02120EB5E4F8F6D8FD756801120ECA26
:10109A0012156B78988673753001C2AF1205AD12BE
:1010AA0005BD1205A31205C41205A31205CB12052C
:1010BA00A31216841205AD1205AD1205A8C2AF78A7
:1010CA00FA79FA308407D9FBD8F7021C00120F36D6
:1010DA00120F6F120FBC120FBD78988673120EB5DD
:1010EA0075881075890275C82475910475D840757C
:1010FA00A82275B80275E690759B80759D0075D11A
:10110A000E75BC5875BB0375BA1175E88012059443
:10111A00D2AF12085D75360053DACF207E0343DA68
:10112A0020307E0343DA1043DA01C2D8C2711205B5
:10113A00ADD2617B037A0CE55B70077A0CDB0302A4
:10114A0010C71205A32070030210C7C270E55CC362
:10115A00940240E1E52F541F855E5DF55EB55DD5CD
:10116A00DAD5C26153DACF207E0343DA20307E0318
:10117A0043DA10C2D8C27178A2E67008D274E52F99
:10118A0054E0F52FC2757529001205A8307409C3F9
:10119A00E529940A4002D275120599780230740240
:1011AA007800C3E55C9840F0C2AF1205BD1205BDD8
:1011BA001205BDD2AF1205AD754C007888E6B403AE
:1011CA000241AA120599788CE6C3940150030212CF
:1011DA00AAE530C3940150030212AA207435C3E56C
:1011EA005C94FF50030212AAC2AF1205D2D2AF1208
:1011FA0005A8C3E55C940150EFC2AF1205BD120504
:10120A009E1205BDD2AF1205A8C3E55C94FF40E962
:10121A000217097F05D27F120FBD1205A8C2AFC2FD
:10122A007F120FBDAE5CC3E55C947FD2AF407B12E8
:10123A000594C2AF1205D2D2AFDFDA120FF4C3EEB1
:10124A0094057897F61205AD1215AD12168C7F0A21
:10125A00D27F120FBD1205A8C2AFC27F120FBDAE58
:10126A005CC3E55C947FD2AF50E4120594C2AF121E
:10127A0005BD12059E1205BDD2AFDFD4120FF4EEE2
:10128A0024037896F61205AD1215AD1216BB120597
:10129A00A8120FBDC3E55C94FF500221E5021709AD
:1012AA00C3E55C954C4003855C4C1205A87801792E
:1012BA0088E7B403027805C3E55C98400221C5C2F9
:1012CA00AF1205D21205D21205D2D2AF1205AD75F0
:1012DA003000E4F531F5320531E531F4703F05327D
:1012EA00789AE67819146012783214600D787D14B1
:1012FA00600878FA146003753200C3E53298401D1D
:10130A00120EB5120594153275310078998673C29A
:10131A00AF1205D2D2AF789886731205A812059E2D
:10132A00E52A700530740201C77801207402780634
:10133A00C3E55C9840A17888E6C39403600312056C
:10134A00A8E52A70030210C7C2AF120EB5E4F5224F
:10135A00F523F524F525F526F567D2AF7885E6C39A
:10136A0033F565E4F544F545F546F547F548F57076
:10137A00F52CF52DF53775700875BB10120594120A
:10138A000861E5E820ECFBA8BDA9BEE97001F88870
:10139A007112086575700875BB10120F36C2AF75E9
:1013AA0061FF1208DD852261852262852263D2AF40
:1013BA0075220175240175250175260185606975F7
:1013CA006A017888E6B40307C27D307602D27DD2FC
:1013DA0068D269753300120E0B120E3C1208FD1208
:1013EA0009041208FD1209041208FD120B7F1206E5
:1013FA00AD120C6D120CB7120904120B6E306E038B
:10140A001206AE206703120800306703120847125B
:10141A000C6D120CE8120904120B7F306E031206CF
:10142A00EA120C6D120D61120904120B6E306E0372
:10143A00120748120C6D120D92120904120B7F301A
:10144A006E031207A5120C6D120E0B120904120874
:10145A0061120B6E120C6D120E3C12086512090411
:0F146A0030692F856461856462856069756A01E8
:1014790079187A0CC3E53399400CC269D26A8A3566
:101489007561FF02149CC3E55C940140030213F5E6
:10149900021522306A1D206C1AE535147006C26ADD
:1014A900D26B61F5F535C3E55C940140030213F590
:1014B900021522753600788279A4E760027803C3A1
:1014C900E55F985054307404E52A604D7888E6B495
:1014D9000317207D0520760781F230760281F220FC
:1014E9006C07D26C856461813478F0306C05856451
:1014F900617820C3E54198500261F5306C1BC26CDC
:10150900C27D307602D27DD26A75351285646161F9
:10151900F50536E55C6002A125753600C2AF120EED
:10152900B57887E6FE7602120F367887EEF6E4F58F
:1015390022F523F524F525F526F565752C00752D7D
:1015490000D2AF1205A8120EB578A4E66006C292C1
:10155900C291C290307409C3E5369404400201C7B0
:1015690041DC901A0D78201215EFE520B45A0CA32E
:101579001215EFE520B4A50302158D120ECA121536
:10158900AD0215AC901A0378807B0A1215EFA308F7
:10159900DBF9901A0F788C7B191215EFA308DBF988
:1015A900901A2822C2AF12162E121608901A007429
:1015B9000E1215F4A374061215F4A374151215F47A
:1015C900901A0378807B0A1215F3A308DBF9901AA5
:1015D9000F788C7B191215F3A308DBF91216411247
:1015E900161F901A2822E493F622E6438F01538F9F
:1015F900FD75EF0275B7A575B7F1F0538FFE22435C
:101609008F02438F0175EF0275B7A575B7F1901A6F
:101619000DF0538FFC22901A0D745AB1F4901A0EE2
:1016290074A5B1F4227A3079D07820901A40B1EFBC
:10163900E520F709A3DAF7227A3079D0901A40E742
:10164900B1F409A3DAF922AB74A875BB0102798454
:10165900BB02027985BB03027986BB04027992BB7E
:1016690005027987BB060279A3BB0702799CBB08EF
:10167900027988BB09027989E8F7227C051205AD50
:10168900DCFB22C2AF1205BD1205C41205CB12053F
:10169900D212059E1205BD1205C41205CB1205D240
:1016A90012059E1205BD1205C41205CB1205D2D230
:1016B900AF22C2AF1205D21205CB1205C41205BD65
:1016C90012059E1205D21205CB1205C41205BD12D0
:1016D900059E1205D21205CB1205C41205BDD2AF63
:1016E90022AE74AF75C2AF1205BD1205BD1205BD9C
:1016F90012059EDEF21205D212059EDFF8D2AF2244
:10170900D18CD184D184757401757501757600D138
:10171900EA7C05AD5C1205ADC3ED955C70F5C3E5DA
:101729005C9401400AC3E55C94FF4032021745D13D
:1017390050B1ADD18CC2AF75EF12D184DCD505762D
:10174900C3E5769403500280C6D1840575E5741407
:1017590090009F93F808C3E57598500280AED18434
:10176900D1840574C3E574940A5002809C120ECA90
:09177900B1ADC2AF75EF12D184CD
:0319FD00021020B5
:101A00000E0615FFFFFFFF03040A0301015AA5019B
:101A1000FFFFFFFFFF03FFFFFF25D0FAFA04FF01DE
:091A2000007AFF0101000300FF40
:101A400023484B696E67323041232020202020201C
:101A500023424C48454C4923463333302320202031
:101A60002020202020202020202020202020202076
:101C0000C2AFC2D353D9BF7581C043B20343FF8073
:101C1000752438752503B1C975EF0275E24043F1AB
:101C20001053A4EF75D4FFD2847DFA780379E67C53
:101C300010752200752300901DD67B0675249875BB
:101C400025013084028142208408D8FBD9F9DCF7D1
:101C500081B4308408D8FBD9F9DCF781B4B189E4C8
:101C600093A3C39A6004DDC381B4DBDBB17B600264
:101C7000812B7B08E493FAA3B15CDBF87A30B15C8A
:101C8000752200752300B17BEAFCEBFDC3ED94FEE9
:101C9000400EB17B8A278B28ED30E0048A828B834B
:101CA000B17B7AC270D8C3ED94FE601350CEBD00F4
:101CB00025EC60097520007521FF0200008100A855
:101CC00027A9280809D804D90281D3B17FEA89AAB3
:101CD000F281C50D81A0C3ED94035049EDA2E092BD
:101CE000007AC5C3E5829400E583941C50902000DF
:101CF00010438F02438F0175B7A575B7F1F030001F
:101D00001FA827A9280809438F01538FFDD804D99C
:101D100002A12089AAE275B7A575B7F1F0A3A10DBC
:101D2000538FFC817C7AC1BD030CE493A3FAB140CC
:101D3000DCF8B138817C817EAA22AB23B15CEBFA5E
:101D4000EA6222752608C3E52313F523E52213F57D
:101D50002250066323A0632201D526EAB1C9B1C986
:101D600075260AEAF4200102D284300102C284B14D
:101D7000C9C3134002C201D526EB22B17FEAFB2082
:101D80008402A17F308402A184752608AE24AF2589
:101D9000C3EF13FFEE13FEB1CDB1C9C3EA13308414
:101DA000024480FA30E703632201C3E52313F523DD
:101DB000E52213F52250066323A0632201D526D91C
:101DC000E52265236523F52222AE24AF250E0FDE22
:101DD000FEDFFCD20122424C48656C693437316326
:041DE000F3300601D5
:00000001FF
